:03000000020800F3
:0C080000787FE4F6D8FD758108020847F7
:030903000108E701
:10088C007590FF758921758CFF758ACE85088DE46E
:10089C00F58BD2AFD2A9D2ABD28CE508F4600905A6
:1008AC00087F0A1208D180031200003094ECE5088E
:1008BC0064CE600915087F0A1208D180031200006B
:0508CC003095EB80D522
:03000B000208E701
:1008E700C28E758CFF758ACE85088DD28EC28132F5
:03001B000208FEDA
:0508FE00C28ED2813220
:0708F700AE071FEE70FA22AC
:1008D100AD071FED600FE4FEEEC394787480948041
:0508E10050EE0E80F353
:0108E60022EF
:10080C0002088CE493A3F8E493A34003F68001F26E
:10081C0008DFF48029E493A3F85407240CC8C333ED
:10082C00C4540F4420C8834004F456800146F6DFBC
:10083C00E4800B0102040810204080900903E47E40
:10084C00019360BCA3FF543F30E509541FFEE493B1
:10085C00A360010ECF54C025E060A840B8E493A378
:10086C00FAE493A3F8E493A3C8C582C8CAC583CAA3
:10087C00F0A3C8C582C8CAC583CADFE9DEE780BE5B
:0109060000F0
:00000001FF
